:020000020000FC
:1000000049CD9CC1000000001FC000008EC0000050
:10001000000098C000000000000000000203040679
:10002000080C10182030406080000406080C1018DE
:100030002030406080A0C00000070F1F3F00050572
:100040000D050205030302004FB662FD0EC05520E8
:1000500009F00994C52DC095089483FDC795C4BDCA
:10006000C093A10064604FBE1895C09164000894CD
:1000700083FDC795C4BDC093A1006B7FC091640090
:10008000CF3F09F41BC04FBE919890989398189554
:1000900091989098939875FD0DC065FD0BC0C9E0CF
:1000A000CA95F1F7C091B300C0FD949AC1FD979A2B
:1000B000C2FD959A2092A1004FBE189524BCCC2772
:1000C000C064C8BF6460F6CFC5CF70FFC3CF65FD05
:1000D000C1CF919ABFCF70FFBDCF65FDBBCF909AC6
:1000E000B9CF70FFB7CF65FDB5CF939AB3CF9498D2
:1000F00070FFB0CF65FDAECFCEE1CA95F1F7919A12
:10010000A9CF979870FFA6CF65FDA4CFCEE1CA9581
:10011000F1F7909A9FCF959870FF9CCF65FD9ACF8D
:10012000CEE1CA95F1F7939A95CF4FB6C9B7CF7E76
:10013000C9BF6E7FCCB5CE0DDDB5DF1DDBBDCABD41
:100140004FBE18953FB68F7EABB7A074A2118061E9
:10015000A0E0ABBFA9B7AE7FA9BF7894A09168001B
:10016000AA2341F085FD2AC0A0916800AA95A0931A
:10017000680024C040E050E085FD14C0A0B396FDA7
:10018000A095A2FD4FEFA3E096FDA2E0A5BFAA2790
:10019000A064AABF8D7FA0B396FDA095A2FD5FEFDE
:1001A000451741F7A8E161FDA093680085FD03C0F4
:1001B000A8E1A093680040939700816085FD0EC080
:1001C000A0916900AA2331F0A0916900AA95A0939B
:1001D000690004C08061AA27A064AABF80FF38C05C
:1001E000A09197004A2F61FF8E7F85FD18C0403F88
:1001F00008F040EFA42FA295AF704A0F5091B800BD
:10020000533069F0A695A69550FD01C0A69552FD04
:1002100003C0A41B4A2F03C04A0F08F44FEFA0915C
:10022000A0004A1708F44A2F40936100A72FA67038
:1002300079F0A0916D00A695A69556E0A50F509176
:100240006100A50FA093610018F4AFEFA0936100C7
:10025000A0916100A093630040916300A0919C0075
:100260004A1708F04A2F542EA091A200AA2309F49D
:1002700022C0542F5A1B10F4A42F50E0BA2E889499
:10028000AA1FAA2EA091A400A095AA22A50E58F0FC
:10029000A091A300A21509F0AA95AA0EA093A3000D
:1002A00048F04A2D08C0A091A300BA1608F0A39503
:1002B000A093A3004FEF40936400A52DA03408F055
:1002C0006860A0916000A395A093600051F0F8943D
:1002D000A9B7A160A9BF84FF02C0A0E4ABBF3FBE25
:1002E0001895A0917400A395A093740041E05091DB
:1002F0006800552329F085FF03C05A955093680084
:10030000A0919700A13018F020929A000DC0209281
:100310009B002092A500A0919A00AF5FA0939A0045
:1003200018F0AFEFA0939A00F894A9B7A160A9BF05
:1003300084FF02C0A0E4ABBF3FBE18953FB64CB5EA
:100340005DB58F7EABB7A074A2118061A0E0ABBF9A
:10035000A9B7AE7FA9BF789481FD23C0A2E096FD26
:10036000A3E0A5BF8260A0B396FDA095A2FF05C043
:1003700040936500509366003EC1A3E096FDA2E065
:10038000A5BFAA27A064AABF8D7F85FF01C026C193
:1003900040E0A0B396FDA095A2FD20C14093970038
:1003A0000FC1A3E096FDA2E0A5BF8D7F61FF71C0E4
:1003B000A2E096FDA3E0A5BFAA27A064AABF826021
:1003C0004093920050939300A09090004A19B090EF
:1003D00091005B09BB24A22C4C38520518F42092E2
:1003E000960049C0A091D600AA2359F1483C520575
:1003F00028F4A0E1BA2EAAE0AA2E23C04836A1E034
:100400005A0728F4A8E0BA2EAFE0AA2E1AC0403D41
:10041000A2E05A0728F4A4E0BA2EAEE1AA2E11C039
:10042000403AA5E05A0728F4A2E0BA2EACE3AA2E7F
:1004300008C04839A8E05A0720F4A1E0BA2EA8E77E
:10044000AA2EC42EA0919400CA1AD52EA091950070
:10045000DA0ADD202AF4AFEFC094D094CA1ADA0A7F
:1004600020929600A8E0A210A0E0CA14DA0618F4C0
:10047000A1E0A09396004093940050939500409182
:10048000920050919300409390005093910002E0AD
:1004900097C0A09165004A1BA09166005A0B94FD7D
:1004A00082C093FD80C092FD7CC086FF03C0D52E24
:1004B000C42E0CC05695479591FD73C0569547952F
:1004C00090FD6FC0D52EC42ED694C79461FD19C07F
:1004D000AC2DAC51AD2DA24008F005C0DD2089F453
:1004E000AC2DA85C70F4A0916700A395AA2311F02D
:1004F000A0936700AA3008F471C020929700816031
:100500006DC0A0916700AA2319F0AA95A093670077
:10051000A22C5091BC0097FD06C0A090CA00533099
:1005200011F4A090D200AAEFAA0EA22DA21DCA1803
:10053000DA0A4FB74170533049F4442321F087FD64
:1005400005C0806803C087FF01C08F77442359F03E
:10055000533031F4AFEFC094D094CA1ADA0A03C012
:1005600040E050E020C0533049F4CC0CDD1CAAE040
:10057000CA1AD20818F4A0E0CA2ED22CAFEFCA16BD
:10058000D20418F04FEF50E00EC0A091AE00CA9E0A
:10059000412D000C441F50E008F012C04FEF50E016
:1005A0000FC05695479594FF07C0552309F04FEFAC
:1005B000A42FA6954A0F521D4F3F520508F04FEF4A
:1005C00040939700816061FF09C0AFE1A095A92326
:1005D000AB299A2F8F7DBB2009F48062A8E1A093FC
:1005E000680085FF03C0AAE0A093680061FD03C016
:1005F00085FD01C08F7E85FD03C0A6E0A093690044
:10060000F894A9B7A160A9BF84FF02C0A0E4ABBF62
:100610003FBE189511E00AC013E008C01AE006C0FA
:100620001EE104C014E602C018EC00C005E1BB27BF
:10063000BA95F1F70A95D9F71A95C1F708952AE303
:1006400038E709C020E33CE806C02AE234EB03C0E7
:1006500025E238EC00C012E095FD9F7D95FF906289
:10066000BB279798BA95F1F7909ABA95F1F79098B9
:10067000BA95F1F7979ABA95F1F7919AB091AF00C0
:10068000BA95F1F79198B7E8BA95F1F71A9521F76D
:10069000022FB22FBA95F1F70A95D9F73A95D9F604
:1006A00097980895221B39E0001F3A9509F40895A0
:1006B000221F211B18F4210F8894F6CF0894F4CF41
:1006C000622C722CB0E08894B395221F331FE0F7A0
:1006D000379527958894912E802E020B130B10F4DA
:1006E000192D082D10F4889401C00894661C771CFD
:1006F000BA9571F7172D062D0895322D11232AF47E
:100700003A9500951095031B130BF894029F712CDA
:10071000002D129F912C802C7894780C172D921C10
:10072000292DB4E06B2E2695179507956A94D9F775
:10073000332321F000951095031B130B08950895A2
:1007400010917B00169500917A000795B0917F007B
:10075000B01B0B2FB0918000B10B1B2F28F4003879
:10076000BFEF1B0740F009C00F37120508F405C0A2
:100770000FE710E002C000E81FEF00938400109321
:100780008500089500918400B09181000B0F1091B5
:100790008500B09182001B1F20E03091850033233B
:1007A0000AF42A95B09183002B1F1AF4203F40F0E1
:1007B0000AC02F3008F407C00FEF1FEF2FE003C06F
:1007C00000E010E020EF30916300B0919C003B17F7
:1007D00018F4323030F009C0B0918500BB235AF0D4
:1007E00004C0B0918500BB2332F4009381001093C4
:1007F00082002093830008952091D8000091840006
:10080000000F10918500111F78DF11232AF40038A2
:10081000BFEF1B0740F009C00F37120508F405C0F1
:100820000FE710E002C000E81FEF002352F0B09184
:100830006200B01B0B2F18F0013008F00AC001E075
:1008400008C000950F5FB09162000B0F08F001C067
:100850000FEF0093860008952091D9000091820047
:10086000109183004ADF11232AF40130BFEF1B07E8
:1008700040F009C00F3F120508F405C00FEF10E06B
:1008800002C001E01FEF112352F0B0918600B01BAF
:100890000B2F18F0013008F00AC001E008C00095E5
:1008A0000F5FB09186000B0F08F001C00FEF0093AF
:1008B000630008950FEF677F71FD29C072FD09C0C5
:1008C0006860B0917B00BA3020F0B52DB03408F4E8
:1008D000677FB091D500BB23D1F0B0917B00BB23E3
:1008E000B1F00FEF10917B00DDDEF894B091730052
:1008F00072FDB5E00B9F112D002D7894112309F0A6
:100900000FEFB0919F000B1710F400919F00009320
:100910009E00089500917A0010917B0000541140D0
:10092000B0919E0010F4BA9501C0B39511F0B09348
:100930009E00089500C008952091B700B6B1B6FD9D
:10094000FBCF04B115B1B6B1BF77B6B9B091AC0069
:10095000B395B093AC00B83060F12092AC00B09188
:10096000D400BB2321F1112329F0B091AD00BF3F8A
:1009700061F009C0B091AD000B1739F020F4BB2332
:1009800021F0BA9502C0B395E1F300919C00B093B9
:10099000AD00B03050F400ECB03038F400E8B030C6
:1009A00020F400E4B03008F400E000939C00777F6E
:1009B0000895B0919C00B39511F0B0939C00B09154
:1009C000AC00B73009F47860089502E3F894B09170
:1009D000DA000B9F012D000C001F7894B0919C0051
:1009E0000B1710F000919C000093610000936300CE
:1009F000502E0093640000939F00089520927A0087
:100A0000B0EFB0937B000895F8940CB51DB520911C
:100A100074007894309175006090760000937500B2
:100A200010937600031B160971FD03C076FD81C08B
:100A30002BC070907700209377002709222311F0B4
:100A40000FEF1FEF8090780090907900309378003E
:100A5000609279006918161910937C000091750056
:100A6000109176000819190920917A0030917B00C5
:100A700036952795020F131F10F40FEF1FEF009309
:100A80007A0010937B0029C020917A0030917B007E
:100A90003901B4E08B2EB2E09B2E343010F08A94F2
:100AA0009A94383010F08A949A94769467948A9441
:100AB000E1F726193709992021F0169507959A94A0
:100AC000E1F7200F311F20937A0030937B0028F448
:100AD0003FEF30937A0030937B00323008F470643B
:100AE00071FF02C0B3E00DC0B091C600009171006B
:100AF000023838F0B395003A08F0B395B63008F0F4
:100B0000B5E09B2EB4E08B2E10917B0000917A0013
:100B100024E0169507952A95E1F70819120928F09F
:100B2000B02FB250B12FB20910F402E010E09801DA
:100B300026C020917A0030917B0039017694679429
:100B40006694669466942619320906950695200FD8
:100B5000321D20937A0030937B00323008F07F7B87
:100B600004E0369527953695279526952695201BE2
:100B700010F0223008F422E089019090C60060FD58
:100B8000FECFE0908C00F0908D006160B9B7B0614D
:100B9000B9BF380176FD44C07694679400938C0009
:100BA00010938D00B92DB330E1F0B0FD04C0060DF7
:100BB000171D930106C0000F111F0250120922E0F9
:100BC00030E0B92DB33068F020938E0030938F0061
:100BD000009388001093890060928A0070928B00C5
:100BE0003DC000938E0010938F00209388003093B7
:100BF000890060928A0070928B0071FF10C0B091E2
:100C00006D00B33060F000918F0010917C0015955D
:100C1000010F28F022F020928E0000938F001EC05A
:100C2000669400938C00B92DB33091F0B0FD03C0F1
:100C3000060D262D03C0000F025022E0B92DB3305F
:100C400038F020938E000093880060928A0006C0DE
:100C500000938E002093880060928A0000917D00AE
:100C600002FD0350013031F495FD0CC0B2E0B06CD0
:100C7000B7B90BC0023021F4B3E0B06CB7B905C00E
:100C800095FDF4CFB4E0B06CB7B90091A400000FAB
:100C900010F4BBE60B270093A40060FDFECFB2E08A
:100CA000B0936E006160B9B7B061B9BFB72FB670CD
:100CB000A1F020917A0030917B0036952795F89429
:100CC0000CB51DB5020F131F1BBD0ABD6160B0E15D
:100CD000B8BFB9B7B061B9BF789408956061209288
:100CE0007E0020E067FD20E206C0606120927E0069
:100CF00020E267FD20E0789401E076FD11C0B72F77
:100D0000B67009F06F7EB0917B00B55048F002E0FC
:100D1000B55020F003E0B55008F006E071FD0AE0A0
:100D200060FD12C0B0917E00BB2371F071FF08C05E
:100D3000B0916D00B33020F0B0916E00BA9519F407
:100D4000789470615CC0AEDF789400000000F89485
:100D500076FD16C010917B00173008F017E0B5E063
:100D60001B0F72FD10E183FF110F62FF110F71FD68
:100D700012E8B4B56090A100B61990F2B10B80F200
:100D8000B0B7B77FB0BFB8B1B0B7B860B0BFB091BF
:100D90007E00B395B0937E00B8B176FD06C0B1E099
:100DA00071FDB2E0BA95F1F7B8B1B072B21709F0BF
:100DB0001BC071FF05C003950A3008F00395B0CF42
:100DC00064FF99CF6F7E3CB56DB470907A008090CF
:100DD0007B00370D681C6BBC3ABD6160B0E1B8BFE9
:100DE000B9B7B061B9BF87CFB0916D00B23008F428
:100DF00082CF64FD80CF0A9509F092CF7F7E20914B
:100E00008E0030918F00F894B0E1B8BF0CB51DB5DD
:100E1000020F131F1BBD0ABDE0908800F0908900EF
:100E20006160B9B7B061B9BF7894B72FB67039F0C7
:100E3000B0916D0072FFB395B0936D0009C074FF5F
:100E400007C067FD05C064FD03C0BF91BF91DEC44C
:100E5000089500E063FF03C064FF01C001E0F8945F
:100E600010917100B7E01B9F212D102D7894200F59
:100E70002695179526951795269517951093710029
:100E8000183718F4B8E7B093710000917100B09171
:100E900072000B1720F0606291989098939860FD13
:100EA000FECFE0908A00F0908B006160B9B7B0612E
:100EB000B9BF0895B2E095FD07C0F894B0937D00E6
:100EC0009798949A7894E5C0F894B0937D00979899
:100ED000959A7894DEC0B3E082FF24C095FD11C0DE
:100EE00002E0F894B0937D00E1E8F0E00093B300F5
:100EF0009398959862FF02C0909A01C0979A78944F
:100F0000C8C002E0F894B0937D00E1E8F0E00093FF
:100F1000B3009198949862FF02C0909A01C0979A8A
:100F20007894B7C095FD0BC0F894B0937D00EBE6C4
:100F3000F0E0939862FF01C0909A7894AAC0F89468
:100F4000B0937D00EBE6F0E0919862FF01C0909ACB
:100F500078949FC0B4E095FD07C0F894B0937D00ED
:100F60009498959A789495C0F894B0937D0095984C
:100F7000949A78948EC0B5E082FF24C095FD11C08C
:100F800001E0F894B0937D00E7E7F0E00093B30050
:100F90009098979862FF02C0919A01C0949A7894B1
:100FA00078C004E0F894B0937D00EBE8F0E00093A3
:100FB000B3009098979862FF02C0939A01C0959AE7
:100FC000789467C095FD0BC0F894B0937D00E5E67A
:100FD000F0E0909862FF01C0919A78945AC0F8941A
:100FE000B0937D00E1E7F0E0909862FF01C0939A32
:100FF00078944FC0B6E095FD07C0F894B0937D009B
:101000009598979A789445C0F894B0937D009498F9
:10101000979A78943EC0B1E082FF24C095FD11C03C
:1010200004E0F894B0937D00EBE8F0E00093B300A7
:101030009198949862FF02C0939A01C0959A78940F
:1010400028C001E0F894B0937D00E7E7F0E000935A
:10105000B3009398959862FF02C0919A01C0949A48
:10106000789417C095FD0BC0F894B0937D00E1E72C
:10107000F0E0919862FF01C0939A78940AC0F894C6
:10108000B0937D00E5E6F0E0939862FF01C0919A8D
:1010900078946F7D089524E630E0F9012092B30042
:1010A0009198909893989498979895986B7F0895B5
:1010B000A4EBB0E00FEF0D930D930D930D9303E0B0
:1010C0000D9304E00D930AE00D9301E00D9301E010
:1010D0000D9301E00D93A0ECB0E001E00D930FEF54
:1010E0000D930D930D930D930D9303E00D930FEF5F
:1010F0000D930FEF0D930D9305E20D9300ED0D93FE
:101100000AEF0D930AEF0D9304E00D930FEF0D938B
:1011100001E00D9300E00D930AE70D930FEF0D939F
:1011200000E00D9301E00D9300E00D9303E00D93BB
:1011300008952091BB008B7FB091BC00B33019F0B3
:101140009F7DB1FD90629F7BB091BD00B1FD906429
:10115000223011F0886001C0877F08950A95E00F62
:10116000F21DB4910895ECE1F0E00091B400F6DFD7
:10117000B093D800ECE1F0E00091B500EFDFB09360
:10118000D900EAE2F0E00091BA00E8DFB093DA00BB
:10119000B091D0000FEF1CE0B23011F400EA1AE079
:1011A000B33011F402E815E000937200109373005D
:1011B000E8E3F0E00091D700D1DFB093A2000895FA
:1011C00008952091CA003091CB00B091BC00B3309B
:1011D00009F43E5097FF02C020E03FEFB32FB21B4F
:1011E0006B2EB25810F4B2E86B2E00E00395609EAF
:1011F000B12DBD57D8F30093AE0008959068E1DF9C
:101200000FDA20E030E0B0E16B2E06DAB091970003
:101210002B0F321D6A94C9F7B4E036952795BA951D
:10122000E1F7822E9F77CDDF0895F894E3E0F0E0B8
:10123000B9E0B7BFB491B078C1F3F894A895B1B54F
:10124000B861B1BDB0E0B1BDB4E0BEBFBFE5BDBFE8
:1012500022DFB0E0B8BBB0E1B7BBB0E0B5BBB0E0F7
:10126000B4BBB0E0B2BBBBEBB1BB2224A0E0B0E0AA
:101270002D92AA31E9F7A0E6B0E00FEF2D920A9582
:10128000E9F7B1E0B093A40013DFF4D2B7E0B06C9B
:10129000B7B9B6B1B460B068B6B90091CC000093EC
:1012A000AF00B1E0B0936A00F894BED9C8D9B8D9FC
:1012B000C9D9B6D9CAD9B4D964D3B6D9B5D9B2D9EE
:1012C000F8940AEF1AEFA0B396FDA095A2FF1FC0F5
:1012D0001A95C9F70A95B1F7E0E0FCE1B591B43E83
:1012E00039F4B591B03E21F4B591BF3F09F40CC07B
:1012F000E0E0F395F395B591B83F49F4B591B43971
:1013000031F4B591BA3A19F4EE27F695099411DF44
:101310002ADF56DF56DF0091CC000093AF00BBDE22
:10132000B2E0B3BFB2E0BEBDB2E0B5BDB1E5B8BF9B
:10133000B9BFB0B7B77FB0BFB8B1B0B7B860B0BFD2
:1013400069D97894F7DAB3E096FDB2E0B5BFB0E4BE
:10135000BBBFBB27B064BABF8D7F66D9626033E084
:101360002CE0B0919600BB2321F42CE03A9509F4CF
:10137000A7CF56D980FFA4CF8E7FB0919700B2300F
:1013800078F3B92FBF710091990000939800B09342
:101390009900B01729F72A9521F76D7FB3E096FDE4
:1013A000B2E0B5BFBB27B064BABF8D7FB091D600A5
:1013B000BB2321F48062B92FB0709B2F8F7B2092CA
:1013C000670030D985FF05C0B0916700BA3008F0DA
:1013D000806422D902E085FF01C000E0B09197004F
:1013E000B017B8F3F8942BD92AD929D978941CD9F5
:1013F00020928700B091BC00B33009F474C00CD9BE
:10140000B091C000B13008F46EC0B0916A00B13044
:1014100008F469C085FD18C0B0919700BF3F08F47B
:1014200062C0F89415D97894FDD8B0919700B13086
:10143000C0F7F89404D9F2D802D97894F3D8B091CF
:101440009700BF3FB0F3CFC2B8E09B2E9068F894EE
:10145000B8DE7894E7D8F8949F77B3DE8090970051
:10146000B0919700BF37789408F445C0D3D8F8946A
:10147000EFD878949A9451F7C1DEB82DB550B09357
:10148000CB00D2D8F89423D281D27894BAE09B2EA4
:101490009068F89496DE7894C5D8F8949F7791DE9A
:1014A00080909700B0919700BF37789478F7B2D8C2
:1014B000F894C5D8B3D8C3D878949A9449F79EDEE7
:1014C000B82DBB5FB093CA00AFD8F89400D26DD2EC
:1014D0007894A8D8F89475DE7894B0919700BF3FBF
:1014E00008F498CF80C200919700B09187000B1745
:1014F00010F00093870096D801E0B091BC00B35083
:1015000009F405E0B0919700B01708F073CFF89494
:101510009FD89ED89DD8789487D820926A00209230
:101520006B0020926C00B0916B00B395B0936B0090
:10153000BF3F69F5B0916C00B395B0936C00B0916A
:10154000CE0009E1BA9559F002E3BA9541F00DE7F2
:10155000BA9529F00AEFBA9511F020926C00B0917B
:101560006C00B017A0F0B0916C00BA95B0936C000D
:10157000B4EBB0936B00B091CD00B093AF00F89492
:1015800067D87894B091CC00B093AF004BD846D8D0
:10159000B0916800BB2319F485FF01C091CE01E032
:1015A00085FD01C006E0B0919700B01708F4BBCFED
:1015B000B091BC00B35009F035D8B0916800BB239E
:1015C00009F47ECEF89467DD2092610020926200DB
:1015D00020926300522C209264002092A300789401
:1015E000B091B900BB0FB093A00020927F00209271
:1015F000800020928100209282002092830020921D
:10160000AC0060E070E020927100B8E0B093AC00F4
:10161000786000D8B7E073FDB7E0B06CB7B9B6B189
:10162000B068B064B6B9B6B1B6FDFDCF04B115B1BE
:10163000B6B1BF77B6B9112309F00FEF0093AD0033
:101640007BD9B8E0B093AC0078608090BB00B2E08A
:10165000B093BB006EDD8092BB00F894BFEFB093F7
:101660009C00B3D9B0916100B0939C00B0939D00F1
:10167000B0939E007894B1E0B0936100B0936300A2
:101680005B2EB0936400B093A600B0919B00B09322
:10169000A500B091BC00B33019F49F7D87FD906226
:1016A0007160726020926D00A5DCB5DCA7D9ACD961
:1016B000A5D9AAD9A3D906C0F8943BDD7894209285
:1016C000AC00777F12DB3BD8C4DBF4DB9DD906DBB3
:1016D00066FD36D876FFEED876FD1CD9BADBFBDB8B
:1016E00093D903DB66FD4ED8B4DB34DC8DD9F6DA52
:1016F00066FD82D8AEDB3FDC87D9F7DA66FDACD871
:10170000A8DB78DC81D9EADAB7E073FDB7E0B06C2A
:10171000B7B9B6B1B068B064B6B99BDB7CDC74D93C
:101720000BD971FF23C067FD21C0B0919F00B0931A
:101730009C00B0939D00B0919B00B093A500B1E0D8
:10174000B093A60018E12CE0B0916D00B11740F005
:101750007D7F746020936F00BFEFB0939C0006C044
:10176000B0919700B13008F0ADCF5AC072FF10C0F1
:1017700067FD0EC0B0916F00BA9511F47B7F9CCFCE
:10178000B0936F00B0919700B13008F09BCF48C084
:1017900020927000B0919A0002E8B01708F040C0A3
:1017A00085FF04C0B0916800BB23D1F1B091BC00AB
:1017B000B33081F495FD03C087FD04C00BC087FFE3
:1017C00001C008C067FD06C06068B0919F00B0937B
:1017D0009C008DCF00EF67FF05C0B0919F00B093D4
:1017E0009C0000E2B0917B00B01708F46BCF67FF5C
:1017F00017C06F779F7D87FD90627460B2E1B093F0
:101800006F00B0919F00B0939C005CCFB0917000CE
:10181000B395B0937000B0919700BB2309F002C05C
:1018200020927000F89437DC8090BB00B2E0B09357
:10183000BB007FDC8092BB0020926100209262009E
:1018400020926300522C209264002092A0007E7FA0
:101850007894E0D620DCB7E0B06CB7B9B6B1B4602C
:10186000B068B6B985FF05C0B0917000B53008F01A
:1018700027CD55CEEDE0F0E023D00A3509F01BC0AE
:10188000EEE0F0E01DD0053A09F015C03AE0A4EB17
:10189000B0E0E3E0F0E014D00D9331963A95D9F73B
:1018A00038E1A0ECB0E0EFE0F0E00AD00D93319623
:1018B0003A95D9F702C0FCDB0AD0E7E2F0E00895E0
:1018C000E199FECFEEBBFFBBE09A0DB308951ED0A9
:1018D0003AE0A4EBB0E0E3E0F0E00D910FD03196F8
:1018E0003A95D9F738E1A0ECB0E0EFE0F0E00D91E7
:1018F00005D031963A95D9F712D00895E199FECFE7
:101900000DBBEEBBFFBBE29AE19A0895EDE0F0E07B
:101910000FEFF4DFEEE0F0E00FEFF0DF0895EDE021
:10192000F0E00AE5EBDFEEE0F0E005EAE7DF08953E
:101930003091B0000091B100313011F40093B80043
:10194000323011F40093B900333011F40093BA002F
:10195000343011F40093C600353011F40093BB000D
:10196000363011F40093D700373011F40093D000D3
:10197000383011F40093BC00393011F40093BD00ED
:10198000089525E051D62A95E9F7089558D65AD6F4
:101990005CD65ED643D653D655D657D659D63ED604
:1019A0004ED650D652D654D6089552D64ED64AD692
:1019B00046D634D64DD649D645D641D62FD648D66A
:1019C00044D640D63CD608958090B0009090B100A7
:1019D00036D635D634D622D68A94D1F739D61ED605
:1019E0009A94E1F70895F894D1DF7894CADFC9DFBB
:1019F000B1E0B093B000B1E0B093B1002092B2007A
:101A0000F894E2DF7894B5E06B2E709097000CD6D6
:101A1000B09197007B16C9F7B13018F0BF3F40F185
:101A200007C086DFF89453DFB1DFB8E0B1BDA9DFAE
:101A30006A9459F7B091B200B395B093B200B33045
:101A400008F4DECF9EDFB091B100B395B093B10042
:101A5000F894B091B000BA95EEE3F0E0EB0FF21D10
:101A6000049178940395B091B100B01708F4C6CFF3
:101A700088DF87DFB091B000B395B093B000B0912C
:101A8000B000BA3008F4B7CF13DBF89420DFB8E029
:061A9000B1BD77DFCACBF7
:00000001FF
